:100000000C9459030C9484030C9484030C9484037F
:100010000C9484030C9484030C9484030C94840344
:100020000C9484030C941D280C9484030C94840376
:100030000C9484030C9484030C9484030C9439155D
:100040000C9484030C9484030C94DA220C9484039F
:100050000C9439250C94CF250C9484030C948403C0
:100060000C9484030C9484030C9484030C948403F4
:100070000C9472250C941C260C9484030C94840319
:100080000C9484030C9484030C948403340EA70F03
:10009000950AA60A000AEE0CA60DAB0AC10A980C36
:1000A0000E0DFC0AE30BAE0B980EF20DEB0A1510C9
:1000B000000A1E0F980EFC0A4E0F850A880AEB0AEA
:1000C000B00FA30F810AC20FBE0F8D0B1D0B930B38
:1000D000400B590BA60D54696E7942617369632018
:1000E000506C75732076302E31340020627974653F
:1000F0007320667265652E0020454550726F6D2035
:10010000627974657320746F74616C2E004F4B00BC
:10011000556E696D706C656D656E74656400486FD1
:10012000773F00576861743F2000536F72727921E6
:1001300000627265616B21004C4953D44C4F41C43D
:100140004E45D75255CE534156C54E4558D44C45D1
:10015000D449C6474F54CF474F5355C252455455C3
:1001600052CE5245CD464FD2494E5055D4505249A9
:100170004ED4504F4BC553544FD04259C546494CAD
:1001800045D34D45CDBFA74157524954C544575259
:100190004954C544454C41D9454EC452534545C4C4
:1001A00043484149CE544F4E45D7544F4EC54E4F0C
:1001B000544F4EC54543484149CE454C4953D4451B
:1001C0004C4F41C445464F524D41D445534156C50D
:1001D0000054CF00535445D00020454550726F6DF8
:1001E00020627974657320617661696C61626C6507
:1001F0002E00484947C848C94C4FD74CCF0008206B
:1002000008003EBD3CBEBEBD3CBDBC21BD0050454E
:1002100045CB4142D341524541C444524541C45269
:100220004EC400060820000000000000000040400E
:1002300040404000400050505000000000000000CE
:1002400050F850F850002070A0702870200000C8AE
:10025000D0205898000020508040A890680040406E
:1002600040000000000010204040402010004020CE
:100270001010102040001038100000000000002076
:1002800020F82020000000000000001010000000F6
:1002900000F800000000000000000010000000084E
:1002A0001020408000007088A8A88870000020609E
:1002B0002020207000007088102040F80000F81006
:1002C000201088700000909090F810100000F880C6
:1002D000F008887000007080F08888700000F808CE
:1002E000102040800000708870888870000070883E
:1002F0008878087000000000200000200000000046
:1003000020002020400000186080601800000000DD
:1003100078007800000000C0300830C00000609015
:10032000202000200000708898A89088700020503D
:1003300088F888880000F088F08888F000007088CD
:10034000808088700000F088888888F00000F8803D
:10035000F88080F80000F880F080808000007088CD
:100360008098887000008888F8888888000070204D
:10037000202020700000381010109060000088903D
:10038000E0A0908800008080808080F8000088D8FD
:10039000A8A8888800008888C8A898880000708865
:1003A000888888700000F088F08080800000708865
:1003B00088A890680000F088F0A0908800007880FD
:1003C000700808F00000F820202020200000888815
:1003D0008888887000008888888850200000888875
:1003E000A8A8A8500000885020508888000088885D
:1003F000502020200000F808102040F80000E08085
:10040000808080E000000080402010080000380854
:10041000080808380000205000000000000000001C
:1004200000000000F80080400000000000000060B4
:100430001070906000008080E09090E0000000006C
:10044000708080700000101070909070000000604C
:1004500090F0807000003040E040404000000060BC
:100460009070101060008080E0909090000020005C
:1004700020202070000010003010101060008090CC
:10048000A0C0A0900000602020202070000000008C
:1004900050A8A8A800000000F0888888000000008C
:1004A00060909060000000006090F080800000008C
:1004B0006090F01010000000B04840400000003094
:1004C0004020106000004040E0404040000000003C
:1004D000909090600000000088885020000000008C
:1004E00088A8A85000000088502050880000000014
:1004F0009090604080000000F02040F0000020401C
:10050000408040402000202020202020200020107B
:1005100010081010200040A810000000000000008B
:1005200000000000000000000000000000000000CB
:10053000000000097E0000000000005121000000C2
:100540005A5341574000004358444524230000209B
:10055000564654522500004E424847595E0000005E
:100560004D4A55262A00003C4B494F292800003EA1
:100570003F4C3A505F00000022007B2B000000003F
:100580000D7D007C00000000000000007F000031B5
:10059000003437000000302E323536381B00002B77
:1005A000332D2A3900000000000000000000000088
:1005B0000000000000000009600000000000007161
:1005C000310000007A73617732000063786465342B
:1005D00033000020766674723500006E62686779B9
:1005E000360000006D6A75373800002C6B696F307B
:1005F0003900002E2F6C3B702D00000027005B3D62
:10060000000000000D5D005C000000000000000024
:100610007F000031003437000000302E323536388C
:100620001B00002B332D2A390000000000000000C1
:100630002100240027002A000000220025002800B5
:100640002B000000200023002600290002020202E5
:100650000202020204040404040404040303030366
:100660000303030301010101010101010102040867
:10067000102040800102040810204080010204087C
:10068000102040800102040810204080000000017A
:100690000200080900000000040307060000000033
:1006A00000000000000000000000000002000E1B1F
:1006B000112711241FBECFEFD0E4DEBFCDBF11E064
:1006C000A0E0B1E0E0EAF7E500E00BBF02C0079070
:1006D0000D92AC32B107D9F71BBE13E2ACE2B1E028
:1006E00001C01D92AD3DB107E1F716E0C2EBD6E0C7
:1006F00004C02297FE010E94932BCE3AD107C9F77E
:100700000E94A7270C94CE2B0C940000CF93DF936C
:10071000BC018230910510F462E070E0A091DB230F
:10072000B091DC23ED01E0E0F0E040E050E021C0DA
:10073000888199818617970769F48A819B81309710
:1007400019F09383828304C09093DC238093DB238E
:10075000FE0134C06817790738F44115510519F0C6
:100760008417950708F4AC01FE018A819B819C01E6
:10077000E9012097E9F641155105A9F1CA01861B47
:10078000970B049708F4BA01E0E0F0E02AC08D91DD
:100790009C91119784179507F9F46417750781F4F4
:1007A00012968D919C911397309719F093838283C1
:1007B00004C09093DC238093DB23FD0132964CC070
:1007C000CA01861B970BFD01E80FF91F6193719316
:1007D00002978D939C9340C0FD01828193819C017F
:1007E000D9011097A1F68091D9239091DA23892B12
:1007F00041F480910201909103019093DA23809358
:10080000D92340910401509105014115510541F44E
:100810004DB75EB78091000190910101481B590BC3
:100820002091D9233091DA23CA01821B930B8617BA
:10083000970780F0AB014E5F5F4F8417950750F02C
:10084000420F531F5093DA234093D923F901619348
:10085000719302C0E0E0F0E0CF01DF91CF91089505
:10086000CF93DF93009709F450C0EC0122971B82CD
:100870001A82A091DB23B091DC23109709F140E0AC
:1008800050E0AC17BD0708F1BB83AA83FE0121919C
:100890003191E20FF31FAE17BF0779F48D919C9150
:1008A0001197280F391F2E5F3F4F398328831296E7
:1008B0008D919C9113979B838A834115510571F407
:1008C000D093DC23C093DB2320C012968D919C91A2
:1008D0001397AD01009711F0DC01D3CFFA01D38358
:1008E000C28321913191E20FF31FCE17DF0769F424
:1008F00088819981280F391F2E5F3F4FFA0131837C
:1009000020838A819B8193838283DF91CF91089595
:10091000A0E0B0E0EEE8F4E00C949F2BEC01A8809E
:10092000B980CA80DB80A114B104C104D10441F4B0
:1009300084E2A82E89EDB82E8BE5C82E87E0D82E4C
:10094000C601B5012DE133EF41E050E00E94762B66
:1009500027EA31E440E050E00E940E2B7B018C013D
:10096000C601B5012DE133EF41E050E00E94762B46
:10097000CA01B9012CEE34EF4FEF5FEF0E940E2B4E
:100980006E0D7F1D801F911F97FF04C06150704046
:1009900080409048688379838A839B839B01AC0164
:1009A0005F77B901CA01CDB7DEB7EAE00C94BB2B83
:1009B0000E948804089586E091E00E9488040895CA
:1009C00060930601709307018093080190930901D9
:1009D00008951F93AC011092C31FA0913E01B091E6
:1009E0003F0160E070E010E004C04F5F5F4F60E0E7
:1009F00070E0FA0124912223A9F1FD01E60FF71F0F
:100A00008081821729F46F5F7F4F4F5F5F4FF1CF77
:100A100090E080589F4F30E082179307A1F4109325
:100A2000C31FFB013196EA0FFB1F01C03196808185
:100A30008032E1F38930D1F3E0933E01F0933F013E
:100A400017C04F5F5F4FFA01849187FFFACF1F5F96
:100A5000FD0101C03196DF0180818032D9F38930F8
:100A6000C9F3C3CF1093C31FB0933F01A0933E01BE
:100A70001F910895482F8091350190913601892B5F
:100A8000E1F48091C41F813089F460913301709149
:100A900034016F5F7F4F7093340160933301615075
:100AA000704083E190E20E94021B08958DE291E084
:100AB000642F40E050E00E94BD1308958AE00E9438
:100AC0003A058DE00E943A050895CF93DF93EC013B
:100AD00005C02196F90184910E943A059E01FE010C
:100AE00084918823B1F7DF91CF9108950E94650525
:100AF0000E945E0508958DE291E061E040ED20EEF8
:100B00000E94CE128DE291E063E272E00E94FD123B
:100B10008CE291E00E94DE1ABC018DE291E00E941D
:100B2000C91286ED90E00E94760583E190E260E0D4
:100B300070E00E94FB1A90E0C0970A97C8F4809179
:100B400037019091380190933A018093390181E007
:100B500080933B01109234011092330181E090E0C8
:100B6000909336018093350190933D0180933C0131
:100B700008950F931F93CF93DF93EC0197FF06C067
:100B8000D095C195DF4F8DE20E943A05E091B51FE7
:100B9000F091B61F00E010E0CE016AE070E00E9424
:100BA000412B805D8293CE016AE070E00E94412B70
:100BB000EB010F5F1F4F1616170674F3F093B61F65
:100BC000E093B51FE091B51FF091B61F8191F093AE
:100BD000B61FE093B51F0E943A050150104091F7EF
:100BE000DF91CF911F910F910895E091C11FF09176
:100BF000C21F808191813396F093C21FE093C11F81
:100C00000E94B90580E20E943A050BC00E943A0595
:100C10008091C11F9091C21F01969093C21F809333
:100C2000C11FE091C11FF091C21F80818A3071F70E
:100C30003196F093C21FE093C11F0E945E05089594
:100C40001F93CF93DF93E0913E01F0913F0101C0EC
:100C50003196DF0190819032D9F39930C9F3F09346
:100C60003F01E0933E019D3261F43196F0933F01E4
:100C7000E0933E010E94200622273327281B390BD0
:100C8000C2C0903331F43196F0933F01E0933E01BE
:100C9000B8C0892F81538930D8F420E030E0C901F1
:100CA00063E0880F991F6A95E1F7220F331F820FC7
:100CB000931F2D9130E020533040280F391F8C9125
:100CC00080538A3060F3B0933F01A0933E019BC0F4
:100CD000892F81548A3108F075C09F012F5F3F4FE3
:100CE000818181548A3198F0892F90E0815490401D
:100CF000880F991FE091B91FF091BA1FE80FF91FF3
:100D00008081918130933F0120933E0148C08EE065
:100D100092E00E94E9041091C31F153009F46EC0DF
:100D2000E0913E01F0913F018081883209F066C078
:100D30003196F0933F01E0933E010E948007EC0161
:100D4000E0913E01F0913F018081893209F056C067
:100D50003196F0933F01E0933E011230C9F0133019
:100D600028F4112341F0113069F50BC01330C9F09C
:100D7000143041F51EC0CF5BDE4F8881282F30E054
:100D800042C09E01D7FF3FC0309521953F4F3BC0E9
:100D90008C2F60E00E9471248C2F0E94D1239C0133
:100DA00032C08C2F60E00E9471248C2F0E94082595
:100DB000F6CFBE01882777FD8095982F0E94E42A00
:100DC0009B0121C0E0913E01F0913F01808188327A
:100DD000A9F43196F0933F01E0933E010E94800711
:100DE0009C01E0913E01F0913F018081893231F414
:100DF0003196F0933F01E0933E0105C081E080937E
:100E0000400120E030E0C901DF91CF911F910895AA
:100E10001F93CF93DF930E942006EC01E0913E01E7
:100E2000F0913F0101C0319680818032E1F3893039
:100E3000D1F3E0933E01F0933F0111E0E0913E01D8
:100E4000F0913F0180818A3281F43196F0933F0125
:100E5000E0933E010E9420069E01289FE001299F09
:100E6000D00D389FD00D1124E9CF8F3291F43196F7
:100E7000F0933F01E0933E010E942006BC010097E1
:100E800029F0CE010E94412BEB01D8CF10934001F5
:100E9000D5CFCE01DF91CF911F910895CF93DF93EE
:100EA000E0913E01F0913F01E081ED3231F0EB3213
:100EB00021F00E940807EC0102C0C0E0D0E0E09100
:100EC0003E01F0913F0180818D3251F43196F093D3
:100ED0003F01E0933E010E940807C81BD90BEFCFEA
:100EE0008B3251F43196F0933F01E0933E010E9422
:100EF0000807C80FD91FE3CFCE01DF91CF91089526
:100F0000CF93DF930E944E07EC018091400188232C
:100F100009F046C082E092E00E94E9048091C31F7C
:100F20008730F1F1833029F1843028F4813099F051
:100F30008230C0F409C0853051F1853008F1863027
:100F400051F0C0E0D0E02CC00E944E0720E0C8174E
:100F5000D90724F122C00E944E0720E0C817D90704
:100F6000E1F41CC00E944E0720E08C179D07B4F4EA
:100F700014C00E944E0720E0C817D90779F40DC0AD
:100F80000E944E0720E08C179D0744F006C00E9487
:100F90004E0720E0C817D9070CF421E0C22FD0E09B
:100FA000CE01DF91CF9108953F924F925F926F9261
:100FB0007F928F929F92AF92BF92CF92DF92EF92E9
:100FC000FF920F931F93CF93DF938FE00E94062829
:100FD00081E491E0909338018093370190933A0136
:100FE0008093390105EB1FE11093B61F0093B51FE5
:100FF00083E89FE19093B81F8093B71F8DE49FE132
:101000009093BA1F8093B91F8CE09EE10E94B905AE
:101010008BEE90E00E94760580E090E10E94B90599
:1010200088EF90E00E947605CC24DD24502E412EDE
:101030001092BC1F1092BB1F5092B51F4092B61F5A
:101040008DE091E00E947605A3E68A2E912CF6E4CD
:101050003F2EE1E06E2EE0E17E2E71E0A72EB12C56
:101060008091BD1F9091BE1F892B29F01092BE1F49
:101070001092BD1F6BC28EE30E943A058091390128
:1010800090913A01029690933F0180933E018091A6
:101090003B01813019F08230B9F422C060913301F4
:1010A000709134016F5F7F4F70933401609333010F
:1010B0006150704083E190E20E94FB1A282F30E0DB
:1010C0002115310569F022C08CE291E00E94BD1A21
:1010D0008823D1F38CE291E00E94CA1A9C0116C0C9
:1010E00010923B01109236011092350180913C0123
:1010F00090913D01892B41F010923D0110923C01ED
:10110000B092BE1FA092BD1F2AE030E02A3049F005
:101110002D3039F0E0913E01F0913F01283009F582
:101120000EC00E945E05E0913E01F0913F018AE011
:101130008083E0913901F0913A0190E03DC08091C7
:10114000390190913A01E817F90709F4A0CF3197D6
:10115000F0933F01E0933E018EEF91E00E9476050F
:1011600096CF8091B91F9091BA1F0297E817F9079F
:1011700011F488E00BC0208380913E0190913F01E3
:10118000019690933F0180933E01822F0E943A0581
:101190007ECF891761F0823269F0873259F0992346
:1011A00041F4813630F08B3720F48052828380E026
:1011B00001C0892F3196982F82818A3051F7809112
:1011C000390190913A01029690933F0180933E013C
:1011D00005C03196F0933F01E0933E01E0913E015E
:1011E000F0913F0180818A30A1F7A091B91FB091A1
:1011F000BA1F1197E0913E01F0913F0180818C93DD
:1012000020913E0130913F018091390190913A0146
:1012100002962817390741F011972150304030933A
:101220003F0120933E01E6CFB0933F01A0933E01E2
:1012300005C03196F0933F01E0933E01E0913E01FD
:10124000F0913F0180818032A1F3893091F320E059
:1012500030E01CC089E12939380718F02FEF3FEF43
:101260001EC0C90163E0880F991F6A95E1F7220F3C
:10127000331F820F931F242F30E020533040280F5C
:10128000391F3196F0933F01E0933E01E0913E011A
:10129000F0913F014081842F80538A30D8F23093FF
:1012A000C01F2093BF1F05C01196B0933F01A093AC
:1012B0003E01A0913E01B0913F018C918032A1F39B
:1012C000893091F38091BF1F9091C01F009709F45E
:1012D000E5C08F5F9F4F09F496C090E001C09F5F0B
:1012E000FD01E90FF11D80818A30C9F7192F1C5FBC
:1012F000FD013397F0933F01E0933E018091BF1FC2
:101300009091C01F918380831283A0913701B09187
:1013100038014091390150913A012091BF1F30911D
:10132000C01FA417B50729F18D919C9111978217C1
:10133000930708F075C612968C911297A80FB11DED
:10134000F0CF12968C911297FD01E80FF11D4E1B04
:101350005F0BED019A0104C08191899321503040C7
:1013600021153105C9F74A0F5B1F50933A0140938D
:101370003901E0913E01F0913F0183818A30E9F526
:101380006FCEE0913901F0913A0180913E01909148
:101390003F018E1B9F0B412F50E08417950708F4E7
:1013A000AC01BF01640F751F9F012A1B3B0BEB01B2
:1013B00004C082918A932150304021153105C9F72C
:1013C000ED0111C0E0913E01F0913F0180818993D0
:1013D00080913E0190913F01019690933F0180934F
:1013E0003E012F5F3F4F2417350760F3141BA40FF6
:1013F000B51F70933A0160933901112311F630CE75
:1014000080E191E002C08EE191E00E94760528CE55
:1014100083E291E00E9465058091BB1F9091BC1F03
:10142000892BC1F0E0913E01F0913F0110811A300B
:1014300011F08EE580838091BB1F9091BC1F90932B
:10144000C21F8093C11F0E94F505E0913E01F091FB
:101450003F0110830E945E0503CE8AE291E03AC00C
:101460003196F0933F01E0933E01E0913E01F0910F
:101470003F0180818A33A1F305C03196F0933F018B
:10148000E0933E01E0913E01F0913F018081803286
:10149000A1F3893091F38A3079F4AEC0E09139013B
:1014A000F0913A013296F0933F01E0933E0132977A
:1014B00082818A3009F4D4CD8CE291E00E94BD1A79
:1014C000882359F08CE291E00E94CA1A4B9729F4C4
:1014D00081E391E00E947605ABCD88E391E00E9424
:1014E000E9048091C31FE82FF0E0E532F10508F030
:1014F00083C0EA5BFF4FEE0FFF1F0590F491E02DD4
:10150000099431E0C32ED12C3DC501E010E0C8C4E0
:10151000109240010E948007AA2797FDA095BA2F3C
:10152000BC01CD010E94302367C0E0913E01F091E3
:101530003F0180818A3009F06BCF80913701909113
:10154000380190933A01809339018ACD8091370117
:10155000909138014CC0109240010E9480079C017C
:1015600080914001882309F04ECFE0913E01F09137
:101570003F0180818A3009F446CF232B09F09CCFAC
:101580003BC0109240010E9480079C019093C01FB5
:101590008093BF1F80914001882309F034CFE091F0
:1015A0003E01F0913F0180818A3009F02CCFE0911B
:1015B0003701F09138014091390150913A01E41717
:1015C000F50721F18081918182179307F8F48281D8
:1015D000E80FF11DF4CFE0913E01F0913F018081D1
:1015E0008A3009F015CF8091390190913A0190939A
:1015F000BC1F8093BB1F0EC0E091BB1FF091BC1FAE
:10160000309709F42DCD8281E80FF11DF093BC1FB6
:10161000E093BB1F2091BB1F3091BC1F809139010B
:1016200090913A012817390709F402CD2D5F3F4FF9
:1016300030933F0120933E013FCFC0E0D0E083E1F3
:1016400090E2BE010E94FB1A482F282F30E021159E
:10165000310591F2C90180978F35910540F02A300C
:10166000310529F02D30310511F08FE301C0842FB1
:101670000E943A05219680E1C030D80701F7BCCF1F
:10168000C0E0D0E0CE018F739070809719F48EE2A5
:101690000E943A0583E190E2BE0140E00E94021BF5
:1016A00021969FE0CF3FD90769F78AE00E943A056B
:1016B000A3CF81E08093C41F1092340110923301B4
:1016C000E0913701F09138014091390150913A0190
:1016D0002091BF1F3091C01FE417F50749F08081AA
:1016E00091818217930720F48281E80FF11DF4CFD6
:1016F000F093C21FE093C11F02C00E94F505209124
:10170000C11F3091C21F8091390190913A01281771
:10171000390799F71092C41F8BCC81E090E0909329
:101720003D0180933C018091370190913801909365
:101730003A0180933901109234011092330181E013
:1017400080933B0181E090E09093360180933501D6
:101750006FCC3196F0933F01E0933E01E0913E0162
:10176000F0913F0190819032A1F3993091F3892F4C
:1017700081548A3108F04CCE3196F0933F01E093CA
:101780003E01E0913E01F0913F0180818032A1F362
:10179000893091F38A3019F08A3309F039CE892FD4
:1017A00090E081549040880F991FE091B91FF0910B
:1017B000BA1FE80FF91F9182808257CE3196F093BD
:1017C0003F01E0933E01E0913E01F0913F01108125
:1017D0001032A1F3193091F3812F81548A3108F02E
:1017E00017CE3196F0933F01E0933E01E0913E0128
:1017F000F0913F0180818032A1F3893091F38D33E4
:1018000009F006CE3196F0933F01E0933E01E0915E
:101810003E01F0913F0180818032A1F3893091F344
:10182000109240010E9480077C0180914001882332
:1018300009F0EECD81ED91E00E94E9048091C31F93
:10184000882309F0E5CD0E948007EC0180914001DA
:10185000882309F0DDCD84ED91E00E94E9048091B8
:10186000C31F882319F041E050E00DC00E9480079B
:10187000AC0180914001882331F0CACD3196F093BC
:101880003F01E0933E01E0913E01F0913F019081E4
:101890009032A1F3993091F39A3019F09A3309F00C
:1018A000B7CD80914001882309F0ADCD9A3009F081
:1018B000AACDA091B51FB091B61F9D01265F3F4FE5
:1018C0008091B71F9091B81F2817390708F4C5CD2C
:1018D0001A97B093B61FA093B51F812F90E0815443
:1018E0009040880F991FE091B91FF091BA1FE80F3F
:1018F000F91FF182E0823C9211961C931197139686
:10190000DC93CE93129715965C934E931497809127
:101910003E0190913F0119969C938E931897809168
:10192000BB1F9091BC1F17969C938E9316979DCDCD
:10193000109240010E9480079093C01F8093BF1FA8
:1019400080914001882309F05ECDE0913E01F09145
:101950003F0180818A3009F056CDE091B51FF091AA
:10196000B61F9F012B5F3F4F8091B71F9091B81F0B
:101970002817390708F471CD3597F093B61FE09317
:10198000B51F87E4808380913E0190913F0194834D
:1019900083838091BB1F9091BC1F92838183E091D0
:1019A0003701F09138014091390150913A0120916D
:1019B000BF1F3091C01FE417F50709F427CE8081BF
:1019C00091818217930708F021CE8281E80FF11DE3
:1019D000F2CF3196F0933F01E0933E01E0913E015A
:1019E000F0913F0180818032A1F3893091F38154DD
:1019F0008A3108F008CD3196F0933F01E0933E0123
:101A0000E0913E01F0913F0180818032A1F3893065
:101A100091F38A3319F08A3009F0FACC8091B51F1E
:101A20009091B61F9093C61F8093C51F85C08C915F
:101A30008634F9F0873409F0FBCA8091C31F8A30DD
:101A4000B1F411968D919C9112979093BC1F809345
:101A5000BB1F13968D919C91149790933F01809397
:101A60003E018091B51F9091B61F05965BC01596FB
:101A70005FC08091C31F853009F059C0E0913E01DD
:101A8000F0913F0131978081282F30E011968C91A1
:101A90001197992787FD90952817390709F047C0B6
:101AA00021543040220F331FE091B91FF091BA1F2B
:101AB000E20FF31F2081318114968D919C9115972F
:101AC000280F391F3183208314968D919C9115978F
:101AD0001816190644F412968D919C91139782174B
:101AE000930754F41AC0892BC1F012968D919C91E2
:101AF0001397281739078CF018968D919C91199798
:101B000090933F0180933E0116968D919C9117977B
:101B10009093BC1F8093BB1FA8CC8091C51F909150
:101B2000C61F0A969093B61F8093B51F9ECC1A9637
:101B3000B093C61FA093C51FA091C51FB091C61F2B
:101B40002FE1A43BB20708F472CF5DCCE0913E01D7
:101B5000F0913F011081812F81548A3108F053CCDC
:101B6000C091B91FD091BA1F3196F0933F01E09315
:101B70003E01E0913E01F0913F0180818032A1F36E
:101B8000893091F38D3309F043CC3196F0933F01C6
:101B9000E0933E01E0913E01F0913F01808180326F
:101BA000A1F3893091F3109240010E9480079C01BB
:101BB00080914001882309F02BCCE0913E01F09107
:101BC0003F01E081EA3019F0EA3309F021CC812F9E
:101BD00090E081549040880F991FC80FD91F398316
:101BE000288343CC109240010E94800780914001DD
:101BF000882331F00DCC3196F0933F01E0933E0104
:101C0000E0913E01F0913F0180818032A1F3893063
:101C100091F38C3209F0FCCB3196F0933F01E093C5
:101C20003E01E0913E01F0913F0180818032A1F3BD
:101C3000893091F3109240010E9480078091400109
:101C4000882309F0E5CBE0913E01F0913F01E0816E
:101C5000EA3009F40ACCEA3309F407CCD9CB31963F
:101C6000F0933F01E0933E01E0913E01F0913F018E
:101C700080818032A1F3893091F320E030E01CC0F4
:101C800089E12939380718F02FEF3FEF1EC0C9014D
:101C9000A3E0880F991FAA95E1F7220F331F820F47
:101CA000931F242F30E020533040280F391F3196E6
:101CB000F0933F01E0933E01E0913E01F0913F013E
:101CC0004081842F80538A30D8F23093C01F2093F4
:101CD000BF1FE0913E01F0913F0180818A3009F001
:101CE00097CBE0913701F091380140913901509143
:101CF0003A01E417F50749F0808191818217930733
:101D000020F48281E80FF11DF4CFF093C21FE0931D
:101D1000C11F02C00E94F5052091C11F3091C21F52
:101D20008091390190913A012817390799F780C9B4
:101D3000E0913E01F0913F01E081EA3361F40E94BD
:101D40005E0580913E0190913F01019690933F0185
:101D500080933E018ACBEA3031F44ECC3196F09339
:101D60003F01E0933E01E0913E01F0913F0110817F
:101D70001032A1F3193091F3123211F0173231F50C
:101D80003196F0933F01E0933E01319703C03196C5
:101D90008A30E1F081818117D1F70BC00E943A05AA
:101DA00080913E0190913F01019690933F01809375
:101DB0003E01E0913E01F0913F018081811771F772
:101DC0003196F0933F01E0933E0118C0E0913E014F
:101DD000F0913F01E081E23209F41ACBE73209F4D5
:101DE00017CB109240010E9480079C018091400116
:101DF000882309F00DCBC9010E94B905E0913E018D
:101E0000F0913F0180818C3209F4A8CF8B3371F4BB
:101E10009F012F5F3F4F81818A3019F08A3309F08B
:101E2000F7CA30933F0120933E011FCB8A3019F04F
:101E30008A3309F0EDCA0E945E0517CB8091B91F65
:101E40009091BA1F2091390130913A01821B930B76
:101E50000E94B9058BEE90E00E94760580E090E14B
:101E60000E94B90588EF90E00E947605C0E0D0E0BE
:101E700083E190E2BE010E94FB1A219690E1C030FE
:101E8000D90711F08823A1F7C3018C1B9D0B0E9479
:101E9000B90589ED91E00E947605E7CA00E010E0FF
:101EA000109240010E948007F82E80914001882303
:101EB00031F0AECA3196F0933F01E0933E01E091DC
:101EC0003E01F0913F0180818032A1F3893091F38E
:101ED0008C3209F09DCA3196F0933F01E0933E01A8
:101EE000E0913E01F0913F0180818032A1F3893081
:101EF00091F382EF91E00E94E9048091C31F843046
:101F000041F0823018F0C0E0D0E00DC0C1E0D0E078
:101F10000AC0109240010E948007EC0180914001AC
:101F2000882309F075CA8F2D61E00E947124012B6E
:101F300029F08F2D6C2F0E94D52497CA8F2DBE01BA
:101F40000E94F32392CAB0923D01A0923C0180917D
:101F500037019091380190933A018093390150CA2A
:101F6000109240010E9480079C01809140018823CB
:101F700009F04ECAC9010E94062B77CA8FE00E9461
:101F8000062873CA109240010E948007EC018091DC
:101F90004001882331F03CCA3196F0933F01E09331
:101FA0003E01E0913E01F0913F0180818032A1F33A
:101FB000893091F38C3209F02BCA3196F0933F01AE
:101FC000E0933E01E0913E01F0913F01808180323B
:101FD000A1F3893091F3109240010E9480079C0187
:101FE00080914001882309F013CA209739F2211506
:101FF000310521F279010027F7FC0095102F8FE0C1
:10200000BE01A80197010E947D28C114D10409F4E2
:102010002CCAC801B7010E943023CC24DD2425CA74
:102020008217930709F0A5C98CC9DF91CF911F9141
:102030000F91FF90EF90DF90CF90BF90AF909F9067
:102040008F907F906F905F904F903F900895FC012C
:10205000613009F1613030F0623009F04BC040E08E
:1020600050E03EC01282138240E050E009C0E0918F
:10207000D81FF091D91FE40FF51F10824F5F5F4FFB
:102080008091D21F2091D31F829FC0011124481735
:1020900059076CF308951282138240E050E03FEF3D
:1020A00009C0E091D81FF091D91FE40FF51F3083CC
:1020B0004F5F5F4F8091D21F2091D31F829FC0013D
:1020C0001124481759076CF30895E091D81FF09137
:1020D000D91FE40FF51F8081809580834F5F5F4F8C
:1020E0008091D21F2091D31F829FC00111244817D5
:1020F00059075CF308952F923F924F925F926F922F
:102100007F928F929F92AF92BF92CF92DF92EF9287
:10211000FF920F931F93DF93CF93CDB7DEB72C972A
:102120000FB6F894DEBF0FBECDBF9A878987A42F64
:1021300029012E2D2C2C462F477078E0F72EF41A0B
:10214000EE2039F4F201E00FF11FE4910F5F1F4F11
:102150002E2F222039F4F201E00FF11FE4910F5FDE
:102160001F4F2E2E822F90E087709070322F369561
:1021700036953695892B29F0822F8770332E33942C
:1021800002C0332E88E0669566956695262F30E06E
:102190003E832D83642E7724B301680F711D8FEF6A
:1021A00090E0AC01062E02C0559547950A94E2F7DF
:1021B00049839C010F2C02C0220F331F0A94E2F7BF
:1021C0002C834B8368507040062E02C095958795EE
:1021D0000A94E2F7685F7F4F8A83CC24DD248A2F3C
:1021E00090E098878F83A32CBB240894A108B108A2
:1021F000A5C02F8138852C0D3D1D8091D31F90E007
:10220000289FD001299FB00D389FB00D1124ED817A
:10221000FE81AE0FBF1FF1E03F1611F4898101C0AE
:1022200080E0E985FA85208131812A0F3B1FF90181
:10223000E080FC818F2B8E21F9018083A201400F69
:10224000511F0F5F1F4FFA013491E985FA85808095
:1022500091808A0E9B1E832F90E0062C02C09595DC
:1022600087950A94E2F7F4012081282B20831196A8
:102270004501800E911E28C0E985FA850190F08104
:10228000E02DEA0FFB1FE080832F90E00F2C02C0AF
:10229000880F991F0A94E2F78083FA013491E98547
:1022A000FA850190F081E02DEA0FFB1F832F90E06B
:1022B000062C02C0959587950A94E2F72081282B79
:1022C000208311960F5F1F4F4F5F5F4F0815190551
:1022D00098F26830710574F41197E985FA85808069
:1022E00091808A0E9B1E1196FB81EF22F401808162
:1022F0008E2980836930710564F0E985FA858080D4
:1023000091808A0E9B1EF4018081FA818F23F40153
:102310008083E985FA85808091808A0E9B1E832FB9
:1023200090E00F2C02C0880F991F0A94E2F7F40185
:102330002081282B20830894C11CD11CC21408F4CE
:1023400058CF2C960FB6F894DEBF0FBECDBFCF91FD
:10235000DF911F910F91FF90EF90DF90CF90BF9092
:10236000AF909F908F907F906F905F904F903F9035
:102370002F900895CF92DF92EF92FF920F931F93C9
:10238000CF93DF93413079F1413038F0423009F496
:1023900054C0433009F0F4C09AC0A091D81FB09146
:1023A000D91F2091D31F30E0862F90E0829FF0014B
:1023B000839FF00D929FF00D1124EA0FFB1F809177
:1023C000D21F90E0829FA001839F500D929F500DDD
:1023D00011244A0F5B1F03C080818D9311924E1709
:1023E0005F07D0F7CDC04091D81F5091D91F2091E1
:1023F000D31F30E08091D21F90E0289FD001299F09
:10240000B00D389FB00D1124A40FB51F862F90E09A
:10241000BC01629FC001639F900D729F900D1124BB
:10242000FD01E81BF90B05C080818C931082119788
:102430003197E417F507C0F7A3C0062F077066951C
:1024400066956695E62EFF2410E0C02FD0E068E088
:1024500070E06C1B7D0B36C02091D31F129FC00112
:102460001124E091D81FF091D91FE80FF91FDF0167
:10247000AE0DBF1D422F50E0425050404E0F5F1F27
:1024800012C030E00C2E02C0220F331F0A94E2F774
:102490001D928C9190E0062E02C0959587950A9426
:1024A000E2F7282B21932C914A175B0750F7822FD4
:1024B00090E0002E02C0880F991F0A94E2F71C9248
:1024C00080831F5F8091D21F181730F259C0062FEA
:1024D0000770669566956695862F90E0EE24FF243A
:1024E000E81AF90A10E0E2E0CE2ED12CC02FD0E09D
:1024F00068E070E06C1B7D0B3EC08091D31F482FBD
:1025000050E09A0121503040189FC0011124280F3B
:10251000391FE091D81FF091D91FE20FF31FDF019F
:10252000AE0DBF1DC601841B950BAC014E0F5F1F86
:1025300013C030E00C2E02C0359527950A94E2F7BF
:102540001C928E9190E0062E02C0880F991F0A946B
:10255000E2F7282B208331972C91A417B50748F771
:10256000822F90E0002E02C0959587950A94E2F79D
:102570001C9280831F5F8091D21F181708F4BDCF73
:10258000DF91CF911F910F91FF90EF90DF90CF904F
:10259000089570930B0160930A010895FF920F93C1
:1025A0001F93CF93DF93EC01F62E022F842F887FA9
:1025B00011F481E01CC0142F169516951695219FD5
:1025C000C00111240E9486039C019983888300978F
:1025D00011F484E00CC01A821B828F2D612F402FD2
:1025E0000E946C14CE0160E00E94271080E0DF9111
:1025F000CF911F910F91FF900895FC017583648323
:102600000895DC0113964C9113971496ED91FC916B
:10261000159731966491242F30E08091D21F90E07D
:10262000861B9109281739072CF0CD0140E00E9444
:10263000BA110895640F13966C930895CF92EF9298
:102640000F931F93DC01022F1496ED91FC911597C7
:10265000329684913197C4903197E490081B0C9D79
:10266000800111240D5F1F4FCD019F010E947B103F
:102670001F910F91EF90CF9008951F93CF93DF9309
:10268000EC01162F6A3069F06B3030F4662309F4E0
:102690003EC06830B9F409C06D3091F06E3091F4ED
:1026A00036C01A820E94011332C0EC81FD81E49190
:1026B0006A816E1B6A834B8120E20E941E1327C031
:1026C0001A8225C06A81EC81FD81E491262F30E0D9
:1026D0008091D31F90E043E0880F991F4A95E1F75E
:1026E0008E1B9109281739073CF01A82CE010E94EF
:1026F0000113CE016A8101C0CE014B81212F0E94BE
:102700001E13EC81FD81E4918A818E0F8A83DF9113
:10271000CF911F910895EF92FF920F931F93CF9344
:10272000DF93EC017A018B012115310521F4642F2F
:102730000E943D131BC02A303105B1F477FF10C051
:102740004DE250E060E070E020E030E00E948B134A
:1027500010950095F094E094E11CF11C011D111DF1
:10276000CE01B801A7012AE00E94D113DF91CF91D9
:102770001F910F91FF90EF900895EF92FF920F93AA
:102780001F93E62E9A01FF24E7FCF0940F2D1F2DD6
:10279000B801A7010E948B131F910F91FF90EF903A
:1027A00008952F923F924F925F926F927F928F92F5
:1027B0009F92AF92BF92CF92DF92EF92FF920F93D0
:1027C0001F93DF93CF93CDB7DEB7A0970FB6F894E2
:1027D000DEBF0FBECDBF1C016A017B014115510553
:1027E0006105710549F440E350E060E070E020E0ED
:1027F00030E00E948B1356C0882499245401422E45
:1028000055246624772401E010E00C0F1D1F080DED
:10281000191DC701B601A30192010E94542BF801B2
:1028200060830894811C911CA11CB11CC701B601D6
:10283000A30192010E94542BC901DA016C017D01B0
:10284000C114D104E104F104F1F651E0E52EF12CBC
:10285000EC0EFD1EE80CF91C3E010894611C711C75
:10286000D501C4010197A109B1096C01C818D908A3
:1028700016C0F601EE0DFF1D40814A3010F4405D98
:1028800001C0495C552747FD5095652F752FC10143
:1028900020E030E00E948B130894E108F1086E14E8
:1028A0007F0439F7A0960FB6F894DEBF0FBECDBFF8
:1028B000CF91DF911F910F91FF90EF90DF90CF901C
:1028C000BF90AF909F908F907F906F905F904F9050
:1028D0003F902F9008950895FF920F931F93F82E25
:1028E000E62F142F3093D91F2093D81F6093D31F46
:1028F0004093D21F1092CB1F1092CC1F1092CD1F6D
:102900001092CE1F882319F084E091E002C088ED78
:1029100090E0612F70E00E94412B61506093D51FC1
:102920000091D51F0093D61F2E2F30E083E0220F99
:10293000331F8A95E1F7442737FD4095542F60EE09
:1029400072E080E090E00E94762B243069F0253020
:1029500018F4233061F410C0253019F0263039F412
:1029600008C087EC96E10AC08DE097E107C02730E8
:1029700018F088E796E102C087E497E19093DB1FA7
:102980008093DA1F0F9A559A17985D9A579A82EC9E
:102990008093800089E180938100412F50E0202FB7
:1029A000332727FD3095FF2011F12F5F3F4F429FC6
:1029B000C001439F900D529F900D112462E070E082
:1029C0000E94412B709561957F4F64566093CF1F95
:1029D00087EC8093D41F87E08093D71F88E391E032
:1029E0009093D11F8093D01F8FEF93E021C02F5F72
:1029F0003F4F429FC001439F900D529F900D112465
:102A000062E070E00E94412B709561957F4F6557A1
:102A10006093CF1F8FEB8093D41F83E08093D71FE9
:102A200086E091E09093D11F8093D01F87EF93E0D1
:102A300090938700809386008AE490E090938900C9
:102A4000809388008091D01F9091D11F0196909320
:102A5000CA1F8093C91F8CEF95E19093DD1F80936F
:102A6000DC1F81E080936F0078941F910F91FF909D
:102A700008951F920F920FB60F920BB60F9211246A
:102A80002F933F934F935F936F937F938F939F9376
:102A9000AF93BF93EF93FF93E0910A01F0910B0185
:102AA0000995E091DC1FF091DD1F0995FF91EF91F1
:102AB000BF91AF919F918F917F916F915F914F9156
:102AC0003F912F910F900BBE0F900FBE0F901F9054
:102AD00018952091C91F3091CA1F8091CF1F90E097
:102AE0002817390779F41092C81F1092C71F8091D8
:102AF000D51F8093D61F82EA95E19093DD1F8093C6
:102B0000DC1F16C02091C91F3091CA1F8091D01FB1
:102B10009091D11F2817390759F48CEF95E19093C4
:102B2000DD1F8093DC1FE0910C01F0910D010995F0
:102B30008091C91F9091CA1F01969093CA1F8093DC
:102B4000C91F0895309184002091D41F2A50231B5F
:102B50002350F0F72D5F19F02A9511F001C0000005
:102B6000E091DA1FF091DB1F09958091D61F882331
:102B700089F48091D51F8093D61F2091D31F809117
:102B8000C71F9091C81F820F911D9093C81F8093FB
:102B9000C71F03C081508093D61F4091C91F509119
:102BA000CA1F4F5F5F4F2091D51F332727FD3095F8
:102BB0002F5F3F4F8091D21F90E0BC01269FC00144
:102BC000279F900D369F900D11242091CF1F820FCB
:102BD000911D4817590731F489E695E19093DD1F5F
:102BE0008093DC1F8091C91F9091CA1F019690931A
:102BF000CA1F8093C91F08952091C91F3091CA1F11
:102C00008091D01F9091D11F281739070CF44EC026
:102C10008CEA93E090938900809388001092CA1FF9
:102C20001092C91F8091CB1F9091CC1FA091CD1FF6
:102C3000B091CE1F0196A11DB11D8093CB1F909323
:102C4000CC1FA093CD1FB093CE1F8091DE1F90911B
:102C5000DF1FA091E01FB091E11F0097A105B10512
:102C600009F18091DE1F9091DF1FA091E01FB091CC
:102C7000E11F181619061A061B0684F58091DE1F3F
:102C80009091DF1FA091E01FB091E11F0197A10972
:102C9000B1098093DE1F9093DF1FA093E01FB093D4
:102CA000E11F1CC01092B1002F9818C02091C91FBD
:102CB0003091CA1F8091D71F992787FD90952817BB
:102CC000390761F48AE490E090938900809388004A
:102CD00089E695E19093DD1F8093DC1F8091C91FE9
:102CE0009091CA1F01969093CA1F8093C91F08959F
:102CF0000F93CF93DF93A091D81FB091D91F8091EC
:102D0000C71F9091C81F2091D31FEC01AC0FBD1FAE
:102D100002B10F7703C000FA07F902B90D90000065
:102D200007FA07F902B900000000000006FA07F9E7
:102D300002B900000000000005FA07F902B900001E
:102D40000000000004FA07F902B9000000000000CA
:102D500003FA07F902B900000000000002FA07F9BF
:102D600002B900000000000001FA07F902B92A9533
:102D700091F60000000000FA07F902B902B10F77DE
:102D800007FB07F902B9DF91CF910F9108950F93D7
:102D9000CF93DF93A091D81FB091D91F8091C71F07
:102DA0009091C81F2091D31FEC01AC0FBD1F02B141
:102DB0000F7703C000FA07F902B90D9007FA07F977
:102DC00002B90000000006FA07F902B9000000008D
:102DD00005FA07F902B90000000004FA07F902B980
:102DE0000000000003FA07F902B90000000002FA2F
:102DF00007F902B900002A9501FA07F902B9D1F6DC
:102E0000000000FA07F902B902B10F7707FB07F9D2
:102E100002B9DF91CF910F9108950F93CF93DF9374
:102E2000A091D81FB091D91F8091C71F9091C81F42
:102E30002091D31FEC01AC0FBD1F02C0000C02B8E3
:102E40000D90000002B800000000000C02B8000065
:102E50000000000C02B800000000000C02B80000E6
:102E60000000000C02B800000000000C02B80000D6
:102E7000000C2A9502B811F70000000C02B80000FF
:102E8000000000001798DF91CF910F9108950F93E4
:102E9000CF93DF93A091D81FB091D91F8091C71F06
:102EA0009091C81F2091D31FEC01AC0FBD1F2E3194
:102EB00091F02D3151F02C3149F02B3141F02A3174
:102EC00039F0293131F0283129F01CC032C048C016
:102ED0005EC074C08AC00D9002B80000000C02B839
:102EE0000000000C02B80000000C02B80000000C4A
:102EF00002B80000000C02B80000000C02B800008C
:102F0000000C02B80D9002B80000000C02B80000DE
:102F1000000C02B80000000C02B80000000C02B85F
:102F20000000000C02B80000000C02B80000000C09
:102F300002B80D9002B80000000C02B80000000CAE
:102F400002B80000000C02B80000000C02B800003B
:102F5000000C02B80000000C02B80000000C02B81F
:102F60000D9002B80000000C02B80000000C02B87E
:102F70000000000C02B80000000C02B80000000CB9
:102F800002B80000000C02B80000000C02B80D905E
:102F900002B80000000C02B80000000C02B80000EB
:102FA000000C02B80000000C02B80000000C02B8CF
:102FB0000000000C02B80000000C02B80D9002B82E
:102FC0000000000C02B80000000C02B80000000C69
:102FD00002B80000000C02B80000000C02B80000AB
:102FE000000C02B80000000C02B80D9002B80000FE
:102FF000000C02B80000000C02B80000000C02B87F
:103000000000000C02B80000000C02B80000000C28
:1030100002B80000000C02B80D9002B80000000CCD
:1030200002B80000000C02B80000000C02B800005A
:10303000000C02B80000000C02B80000000C02B83E
:103040000000000C02B80D9002B80000000C02B89D
:103050000000000C02B80000000C02B80000000CD8
:1030600002B80000000C02B80000000C02B800001A
:10307000000C02B80D9002B80000000C02B800006D
:10308000000C02B80000000C02B80000000C02B8EE
:103090000000000C02B80000000C02B80000000C98
:1030A00002B80D9002B80000000C02B80000000C3D
:1030B00002B80000000C02B80000000C02B80000CA
:1030C000000C02B80000000C02B80000000C02B8AE
:1030D0000D9002B80000000C02B80000000C02B80D
:1030E0000000000C02B80000000C02B80000000C48
:1030F00002B80000000C02B80000000C02B80D90ED
:1031000002B80000000C02B80000000C02B8000079
:10311000000C02B80000000C02B80000000C02B85D
:103120000000000C02B80000000C02B80D9002B8BC
:103130000000000C02B80000000C02B80000000CF7
:1031400002B80000000C02B80000000C02B8000039
:10315000000C02B80000000C02B80D9002B800008C
:10316000000C02B80000000C02B80000000C02B80D
:103170000000000C02B80000000C02B80000000CB7
:1031800002B80000000C02B80D9002B80000000C5C
:1031900002B80000000C02B80000000C02B80000E9
:1031A000000C02B80000000C02B80000000C02B8CD
:1031B0000000000C02B80D9002B80000000C02B82C
:1031C0000000000C02B80000000C02B80000000C67
:1031D00002B80000000C02B80000000C02B80000A9
:1031E000000C02B80D9002B80000000C02B80000FC
:1031F000000C02B80000000C02B80000000C02B87D
:103200000000000C02B80000000C02B80000000C26
:1032100002B80D9002B80000000C02B80000000CCB
:1032200002B80000000C02B80000000C02B8000058
:10323000000C02B80000000C02B80000000C02B83C
:103240000D9002B80000000C02B80000000C02B89B
:103250000000000C02B80000000C02B80000000CD6
:1032600002B80000000C02B80000000C02B80D907B
:1032700002B80000000C02B80000000C02B8000008
:10328000000C02B80000000C02B80000000C02B8EC
:103290000000000C02B80000000C02B80D9002B84B
:1032A0000000000C02B80000000C02B80000000C86
:1032B00002B80000000C02B80000000C02B80000C8
:1032C000000C02B80000000C02B80D9002B800001B
:1032D000000C02B80000000C02B80000000C02B89C
:1032E0000000000C02B80000000C02B80000000C46
:1032F00002B80000000C02B80D9002B80000000CEB
:1033000002B80000000C02B80000000C02B8000077
:10331000000C02B80000000C02B80000000C02B85B
:103320000000000C02B80D9002B80000000C02B8BA
:103330000000000C02B80000000C02B80000000CF5
:1033400002B80000000C02B80000000C02B8000037
:10335000000C02B80D9002B80000000C02B800008A
:10336000000C02B80000000C02B80000000C02B80B
:103370000000000C02B80000000C02B80000000CB5
:1033800002B80D9002B80000000C02B80000000C5A
:1033900002B80000000C02B80000000C02B80000E7
:1033A000000C02B80000000C02B80000000C02B8CB
:1033B0000D9002B80000000C02B80000000C02B82A
:1033C0000000000C02B80000000C02B80000000C65
:1033D00002B80000000C02B80000000C02B80D900A
:1033E00002B80000000C02B80000000C02B8000097
:1033F000000C02B80000000C02B80000000C02B87B
:103400000000000C02B80000000C02B80D9002B8D9
:103410000000000C02B80000000C02B80000000C14
:1034200002B80000000C02B80000000C02B8000056
:10343000000C02B80000000C02B800000000179851
:10344000DF91CF910F9108958091C00087FF13C045
:103450009091E21F9F5F9D3208F090E08091E31F02
:10346000981749F08091C600E92FF0E0EA51F04E3C
:1034700080839093E21F08954091E21F2091E51F01
:103480003091E31F341759F03F5F3D3208F030E0D0
:10349000E32FF0E0EA51F04EE081EE2331F4209387
:1034A000E51F3093E31F80E00895E03F11F42160B1
:1034B000E9CFE03E11F42260E5CF822F90E020FFBB
:1034C00009C0E23111F42B7F03C0E93509F4277FED
:1034D0002C7FD8CFE23111F42460D4CFE93511F438
:1034E0002860D0CF21FF2DC0E23719F1E33760F417
:1034F000EA3529F1EB3518F4EA34A9F51EC0EB36AC
:10350000B1F0E13781F50DC0E53779F0E63718F411
:10351000E43749F510C0EA3731F0ED3721F589E19C
:1035200023C08FE721C08AE11FC08BE01DC088E067
:103530001BC08AE019C085E117C08FE215C08DE07D
:1035400013C08C709070892B39F0E43860F4F0E08F
:10355000EA5DFA4F849108C0E43828F4F0E0E655BB
:10356000FA4F849101C080E02C7F882309F48ACF30
:103570002093E51F3093E31F08958091E41F882373
:1035800011F081E008950E943C1A8093E41F81119C
:1035900081E008958091E41F882319F01092E41FC0
:1035A00007C00E943C1A882319F42FEF3FEF04C094
:1035B000282F332727FD3095C90108951092C000A8
:1035C00083E390E09093C5008093C40088E18093EA
:1035D000C100E2ECF0E080818064808380818062C1
:1035E00080838081806180831092E21F1092E31FAC
:1035F00084E29AE10895F999FECF72BD61BDF89A0F
:1036000080B50895F999FECF1FBA72BD61BD40BD66
:103610000FB6F894FA9AF99A0FBE089510921920ED
:1036200010921A2010921D2010921F2082E090E02C
:10363000A0E0B0E08093202090932120A09322204E
:10364000B0932320109237201092412010924020F6
:1036500088E191E090933F2080933E201092432098
:103660000895FF920F931F93CF93DF938B010E94D6
:103670002223EB01FF24FA94FEBC0DB407FEFDCF1C
:103680008EB58F3F11F481E008C00E9422236C1B8D
:103690007D0B6017710780F380E0DF91CF911F9160
:1036A0000F91FF900895FC01848160E00E94D52471
:1036B0000895FC01848161E00E94D5240895DC0115
:1036C0006EBDFA0120E030E00DB407FEFDCF808131
:1036D0008EBD0DB407FEFDCF81818EBD2E5F3F4FA5
:1036E000329682E02030380779F70DB407FEFDCF1F
:1036F0008FEF8EBD0DB407FEFDCF8FEF8EBD0DB4E5
:1037000007FEFDCF8FEF8EBD0DB407FEFDCF8EB54A
:103710001A968C931A978F71853011F481E0089571
:1037200081E115968C931597CD010E94591B80E07D
:103730000895FF920F931F93CF93DF93EC010E94A4
:1037400022238B01FF24FA9409C00E942223601BCC
:10375000710B6D52714010F08FE00DC0FEBC0DB4C6
:1037600007FEFDCF8EB58A878F3F79F38E3F11F428
:1037700081E006C08DE08D83CE010E94591B80E060
:10378000DF91CF911F910F91FF900895CF93DF9319
:10379000EC018E818823D1F08FEF8EBD2F8138858B
:1037A0004FEF04C00DB407FEFDCF4EBD2F5F3F4F5E
:1037B000C901019781509240A8F338872F830DB437
:1037C00007FEFDCFCE010E94591B1E82DF91CF91D3
:1037D0000895DF92EF92FF920F931F93CF93DF93A1
:1037E000EC01D62E79018A010E94C61BCE010E94EF
:1037F000531BCE016CE271E00E94311B8D2D806461
:103800008EBD0DB407FEFDCF28E130E0D801C70121
:10381000022E04C0B695A795979587950A94D2F77E
:103820008EBD0DB407FEFDCF285030408FEF283FEE
:10383000380761F7DD2011F485E906C088E0D81665
:1038400011F487E801C08FEF8EBD0DB407FEFDCFE8
:1038500090E02FEF2EBD0DB407FEFDCF8EB587FF94
:1038600002C09150B9F78A87DF91CF911F910F91D4
:10387000FF90EF90DF900895CF92DF92EF92FF924A
:103880000F931F93CF93DF93EC017A018B016901B2
:10389000411551056105710511F482E137C08B8531
:1038A000833039F029E0EE0CFF1C001F111F2A9510
:1038B000D1F7CE0168E1A80197010E94E91B882396
:1038C00011F084E023C0CE016EEFA6010E945F1BC1
:1038D0008823E9F0CE0168E572E00E94311B88235D
:1038E00011F485E113C0CE016DE020E030E040E04E
:1038F00050E00E94E91B882341F48FEF8EBD0DB488
:1039000007FEFDCF8EB5882379F084E18D83CE014B
:103910000E94591B80E0DF91CF911F910F91FF9082
:10392000EF90DF90CF900895CE010E94591B81E067
:10393000F2CF8F929F92AF92BF92CF92DF92EF928F
:10394000FF920F931F93CF93DF93EC015A016B010A
:1039500049010115110509F47BC0C801820F931FAD
:103960008150924008F06FC08E81882371F0888169
:103970009981AA81BB81481759076A077B0729F4F7
:103980008F8198858816990618F5A882B982CA820F
:10399000DB828B85833039F069E0AA0CBB1CCC1C20
:1039A000DD1C6A95D1F7CE0161E1A60195010E9467
:1039B000E91B882319F083E08D8345C0CE010E9466
:1039C000991B882309F43FC018861F8281E08E83EB
:1039D0008FEF8EBD8F8198852FEF05C00DB407FE48
:1039E000FDCF2EBD019688159905C0F398878F836A
:1039F000D801119720E030E09FEF0BC00DB407FE17
:103A0000FDCF8EB5F701E20FF31F80839EBD2F5FC0
:103A10003F4F2A173B0790F30DB407FEFDCF8EB53D
:103A2000AE0DBF1D8C932F813885200F311F388735
:103A30002F838985882319F02050324048F0CE0129
:103A40000E94C61B05C0CE010E94591B80E001C028
:103A500081E0DF91CF911F910F91FF90EF90DF9068
:103A6000CF90BF90AF909F908F900895EF92FF926C
:103A70000F931F93790120E030E000E012E00E94F4
:103A8000991C1F910F91FF90EF9008956F927F9274
:103A90008F929F92AF92BF92CF92DF92EF92FF925E
:103AA0000F931F93CF93DF93EC017A018B012D814C
:103AB000222309F480C08B899C89AD89BE89841733
:103AC0009507A607B70708F476C085C0E114F1048E
:103AD0000105110549F41E821F82188619861A866F
:103AE0001B861C861D8665C02A853B854C855D85A9
:103AF000EB8DFC8D858590E009962150304040404B
:103B0000504039014A01082E04C096948794779456
:103B100067940A94D2F72F5F3F4F4F4F5F4F08943F
:103B2000E108F108010911095701680104C0D694A0
:103B3000C794B794A7948A95D2F70894E11CF11C16
:103B4000011D111DA614B704C804D90428F02115BD
:103B500031054105510549F48F89988DA98DBA8D9C
:103B60008E839F83A887B98716C0A618B708C80890
:103B7000D90811C04E815F81688579858B8D9C8DB8
:103B800094010E9458210894A108B108C108D108E5
:103B9000882331F410C086E0882E912C8C0E9D1E57
:103BA000A114B104C104D10429F7EA86FB860C876D
:103BB0001D8781E001C080E0DF91CF911F910F91BF
:103BC000FF90EF90DF90CF90BF90AF909F908F903D
:103BD0007F906F900895223009F078CFE6CFCF9391
:103BE000DF93EC01462F6E857F85888999890E9435
:103BF0008120882319F420E030E00AC08A89282F28
:103C000030E095E0220F331F9A95E1F7215A3F4D9E
:103C1000C901DF91CF9108950F931F93CF93DF9345
:103C20008C01FC0185818823D9F1848187FF35C00F
:103C3000C80161E00E94EF1DEC01009789F1F801D5
:103C40008581823040F483899489A589B6898C8FD7
:103C50009D8FAE8FBF8FF8018789908D9B8F8A8F44
:103C60008789908DA18DB28DCD01AA27BB279D8B11
:103C70008C8BE0915D20F0915E20309751F0BE0179
:103C80006A5E7F4FCE0148960995888D998D9B8BF2
:103C90008A8BF80184818F7784830E94462001C03B
:103CA00080E0DF91CF911F910F910895CF93DF9323
:103CB000EC019C012A5F3F4F8B8D9C8D41E050E0D1
:103CC00060E070E00E94CB218823A1F08F89988D5D
:103CD000A98DBA8D0097A105B10559F48E819F81F8
:103CE000A885B9858F8B988FA98FBA8F8C818068B2
:103CF0008C8381E0DF91CF9108952F923F924F9274
:103D00005F927F928F929F92AF92BF92CF92DF92FB
:103D1000EF92FF920F931F93DF93CF9300D000D0C9
:103D200000D0CDB7DEB76C01162F072F5E834D8311
:103D3000DC0115968C911597813009F070C11496AD
:103D40008C9181FF6CC18EC1F601438954896589CC
:103D5000768982859385A485B58584179507A607FE
:103D6000B70731F0C6010E94461D882309F457C1E8
:103D7000812F902F9C0129012D803E8017C1D601F3
:103D80005B96ED91FC915C97DA01C90119E0B6955B
:103D9000A795979587951A95D1F774807A9478228C
:103DA0007FEF872E71E0972E82229322772009F0F1
:103DB0004EC08114910409F04AC0D60116964D9167
:103DC0005D916D917C9119974115510561057105C2
:103DD00081F457968D919D910D90BC91A02D0097E7
:103DE000A105B10549F1F60186839783A087B187C4
:103DF0002EC0CF019E012F5F3F4F0E945821882384
:103E000009F414C129813A814B815C81D6015B960A
:103E1000ED91FC915C978789803129F088EF9FEFC5
:103E2000AFEFBFE004C088EF9FEFA0E0B0E028173D
:103E300039074A075B0730F0C6010E94561E8823E7
:103E400031F4EDC0F601268337834087518780E047
:103E500092E08819990951018215930508F45C01D3
:103E6000D6015B96ED91FC915C971696ED90FD90D6
:103E70000D911C9119978EEF9FEFAFEFBFEFE80EFA
:103E8000F91E0A1F1B1F058404C0EE0CFF1C001F37
:103E9000111F0A94D2F786859785A089B189E80E0B
:103EA000F91E0A1F1B1FE70CF11C011D111D90E0DC
:103EB000A91692E0B90651F580910E0190910F017B
:103EC000A0911001B09111018E159F05A007B107B7
:103ED00061F48FEF9FEFAFEFBFEF80930E019093F0
:103EE0000F01A0931001B093110180915F22909176
:103EF0006022B801A70192010E943C1C882309F4AA
:103F00008EC0A0E0B2E04A0E5B1E3EC08114910458
:103F100009F5F60122853385448555858389948981
:103F2000A589B689281739074A075B0798F00E94C8
:103F30004620882309F473C0E0920E01F0920F012D
:103F40000093100110931101809161228160809390
:103F5000612208C0C801B70141E00E948120882386
:103F600009F45DC09401215A3F4DA9014A0D5B1D22
:103F7000D201F90102C08D918193E417F507D9F7B9
:103F8000E21BF30B4E0E5F1E2A183B08950140E022
:103F900050E0F60182859385A485B585820F931F35
:103FA000A41FB51F82879387A487B587D6011A9669
:103FB0002D913D914D915C911D972114310409F093
:103FC000DECE53968D919D910D90BC91A02D8217C0
:103FD0009307A407B50748F4F601238B348B458B70
:103FE000568B84818068848311C080915D2090917C
:103FF0005E20892B59F08D819E81892B39F0D60165
:1040000014968C911497806814968C93F601848191
:1040100083FF0EC0C6010E940C1E882349F481E074
:1040200090E0D60113969C938E9312971E821D8268
:104030008D819E8126960FB6F894DEBF0FBECDBF50
:10404000CF91DF911F910F91FF90EF90DF90CF9074
:10405000BF90AF909F908F907F905F904F903F90D8
:104060002F90089582FD70CE83CEDF93CF930F9271
:10407000CDB7DEB76983BE016F5F7F4F41E050E08F
:104080000E947D1E0F90CF91DF9108958091612253
:10409000882399F140910E0150910F016091100118
:1040A0007091110180915F22909160222FE530E2A2
:1040B0000E943C1C882319F1409162225091632296
:1040C0006091642270916522411551056105710569
:1040D00091F080915F22909160222FE530E20E9462
:1040E0003C1C882361F0109262221092632210928D
:1040F0006422109265221092612281E0089580E08E
:104100000895DF92EF92FF920F931F937B018C0132
:10411000D42E80910E0190910F01A0911001B091C9
:1041200011018E159F05A007B107C1F00E9446201E
:104130008823D9F080915F2290916022B801A70175
:104140002FE530E20E94361D882379F0E0920E01BF
:10415000F0920F01009310011093110180916122E0
:104160008D298093612281E001C080E01F910F9131
:10417000FF90EF90DF9008954F925F926F927F9241
:104180008F929F92AF92BF92CF92DF92EF92FF9267
:104190000F931F93CF93DF93EC016A017B012801FA
:1041A0003901423051056105710508F46FC08985F8
:1041B0009A85AB85BC850196A11DB11D8417950715
:1041C000A607B70708F462C02B893C894D895E8930
:1041D0008F89803129F499278F2D7E2D6D2D09C06F
:1041E000C701B60117E096958795779567951A955B
:1041F000D1F74B015C01820E931EA41EB51E809167
:104200000E0190910F01A0911001B091110188163B
:104210009906AA06BB0639F0C501B40140E00E9428
:104220008120882399F18F89803149F4F601F0705B
:10423000EE0FFF1FE15AFF4D518240820DC0F60183
:10424000EF77F070EE0FFF1FEE0FFF1FE15AFF4DEB
:104250004082518262827382809161228160809368
:1042600061228A89823080F08D819E81AF81B885FC
:10427000880E991EAA1EBB1E809262229092632213
:10428000A0926422B092652281E001C080E0DF91BB
:10429000CF911F910F91FF90EF90DF90CF90BF9043
:1042A000AF909F908F907F906F905F904F90089508
:1042B000CF92DF92EF92FF920F931F93CF93DF93F2
:1042C000EC017A018B01690189859A85AB85BC85F2
:1042D0000196A11DB11D84179507A607B70708F41D
:1042E00050C02B893C894D895E898F89803129F4A2
:1042F0009927812F702F6F2D09C0C801B701E7E002
:104300009695879577956795EA95D1F7260F371F8C
:10431000481F591F80910E0190910F01A09110012B
:10432000B0911101281739074A075B0739F0CA0114
:10433000B90140E00E948120882319F18F898031E2
:1043400059F4F701F070EE0FFF1FE15AFF4D808125
:104350009181A0E0B0E00EC0F701EF77F070EE0FB2
:10436000FF1FEE0FFF1FE15AFF4D80819181A28157
:10437000B381BF70F60180839183A283B38381E010
:1043800001C080E0DF91CF911F910F91FF90EF90DE
:10439000DF90CF9008952F923F924F925F926F924D
:1043A0007F928F929F92AF92BF92CF92DF92EF92C5
:1043B000FF920F931F93DF93CF93CDB7DEB72F9765
:1043C0000FB6F894DEBF0FBECDBF1C014A875B87D6
:1043D0006C877D873F872E87D9010D911D912D9187
:1043E0003C91011511052105310549F0480159019C
:1043F0000894811C911CA11CB11C198610C0FC01E1
:1044000080809180A280B38019868A859B85AC8547
:10441000BD850197A105B10511F491E09987D101FE
:1044200019968D919D910D90BC91A02D0196A11D85
:10443000B11D8D839E83AF83B887750164014424C9
:10444000552432018E010F5F1F4FF1018185928546
:10445000A385B485481659066A067B0608F090C005
:104460008D819E81AF81B8858C159D05AE05BF05F8
:1044700050F482E0882E912CA12CB12CB2E0CB2EEE
:10448000D12CE12CF12CC101B701A60198010E94A9
:104490005821882309F474C089819A81AB81BC8139
:1044A000A70196012F5F3F4F4F4F5F4F0097A10528
:1044B000B10519F049015A010DC0281939094A09F5
:1044C0005B098A859B85AC85BD85281739074A0716
:1044D0005B0759F00894411C511C611C711C089425
:1044E000C11CD11CE11CF11CB0CFC101A601B70158
:1044F0000FEF1FEF2FEF3FE00E94BC20882399F4BD
:104500003FC026013701089441085108610871082D
:10451000C101B301A201970186010E94BC2088233A
:1045200079F1730162018C149D04AE04BF0448F359
:10453000AE85BF854D915D916D917C914115510581
:104540006105710539F0C101950184010E94BC200B
:104550008823B1F0EE85FF8580829182A282B382AA
:10456000F985FF2359F00894811C911CA11CB11CF2
:10457000D1018D929D92AD92BC92139781E001C0C2
:1045800080E02F960FB6F894DEBF0FBECDBFCF915F
:10459000DF911F910F91FF90EF90DF90CF90BF9030
:1045A000AF909F908F907F906F905F904F903F90D3
:1045B0002F9008951F920F920FB60F9211242F93F0
:1045C0003F938F939F93AF93BF9380916A22909173
:1045D0006B22A0916C22B0916D2230916E220196D7
:1045E000A11DB11D232F2D5F2D3720F02D570196D2
:1045F000A11DB11D20936E2280936A2290936B229D
:10460000A0936C22B0936D228091662290916722D4
:10461000A0916822B09169220196A11DB11D8093DD
:10462000662290936722A0936822B0936922BF917B
:10463000AF919F918F913F912F910F900FBE0F904F
:104640001F9018958FB7F89420916A2230916B22B1
:1046500040916C2250916D228FBFB901CA0108951B
:104660009B01AC017FB7F8948091662290916722FC
:10467000A0916822B091692266B5A89B05C06F3FE2
:1046800019F00196A11DB11D7FBFBA2FA92F982F38
:104690008827860F911DA11DB11D62E0880F991F0B
:1046A000AA1FBB1F6A95D1F7BC012DC0FFB7F894B4
:1046B0008091662290916722A0916822B091692230
:1046C000E6B5A89B05C0EF3F19F00196A11DB11DED
:1046D000FFBFBA2FA92F982F88278E0F911DA11DDC
:1046E000B11DE2E0880F991FAA1FBB1FEA95D1F701
:1046F000861B970B885E9340C8F2215030404040A3
:10470000504068517C4F211531054105510571F626
:104710000895789484B5826084BD84B5816084BD39
:1047200085B5826085BD85B5816085BDEEE6F0E02A
:10473000808181608083E1E8F0E010828081826086
:104740008083808181608083E0E8F0E08081816007
:104750008083E1EBF0E0808184608083E0EBF0E037
:10476000808181608083E1E9F0E0808182608083E4
:10477000808181608083E0E9F0E0808181608083D6
:10478000EAE7F0E0808184608083808182608083BA
:104790008081816080838081806880831092C100E5
:1047A0000895982F883108F09851977080911201E0
:1047B0008295880F880F807C892B80937C00809164
:1047C0007A00806480937A0080917A0086FDFCCF25
:1047D0002091780040917900942F80E030E0282BE0
:1047E000392BC90108951F93CF93DF93182FEB0145
:1047F00061E00E947124209709F468C0CF3FD10581
:1048000009F467C0E12FF0E0E457F94F8491843058
:1048100061F1853040F48230C9F08330E0F48130BA
:1048200009F051C00EC0873091F1883020F48630F5
:1048300009F049C024C0883091F1893009F043C0A3
:1048400038C084B5806884BDC7BD47C084B5806268
:1048500084BDC8BD42C08091800080688093800084
:10486000D0938900C093880038C080918000806216
:1048700080938000D0938B00C0938A002EC08091DB
:10488000B00080688093B000C093B30026C08091D0
:10489000B00080628093B000C093B4001EC08091CD
:1048A0009000806880939000D0939900C093980006
:1048B00014C080919000806280939000D0939B0000
:1048C000C0939A000AC0C038D1051CF4812F60E063
:1048D00002C0812F61E00E94D524DF91CF911F910A
:1048E0000895482F50E0CA018459994FFC01249142
:1048F000445B594FFA0184918823C1F0E82FF0E01E
:10490000EE0FFF1FE25DF94FA591B491662341F4CC
:104910009FB7F8948C91209582238C939FBF089524
:104920009FB7F8948C91822B8C939FBF089584300D
:10493000C9F0853038F48230F1F0833078F481307A
:1049400099F516C08730F9F0883018F4863061F593
:1049500016C08830F1F0893039F521C0809180008F
:104960008F7703C0809180008F7D809380000895B1
:1049700084B58F7702C084B58F7D84BD0895809102
:10498000B0008F7703C08091B0008F7D8093B0001E
:104990000895809190008F77809390000895809182
:1049A00090008F7D809390000895FF920F931F9346
:1049B000F62E482F50E0CA018457994FFC012491EC
:1049C000CA018459994FFC011491445B594FFA0173
:1049D00004910023C9F0222319F0822F0E9497240A
:1049E000E02FF0E0EE0FFF1FE85CF94FA591B491C6
:1049F0009FB7F894FF2021F48C911095812302C079
:104A00008C91812B8C939FBF1F910F91FF900895E4
:104A10000F931F93482F50E0CA018457994FFC0110
:104A20002491CA018459994FFC010491445B594F68
:104A3000FA011491112319F420E030E015C022236B
:104A400019F0822F0E949724812F90E0880F991FE0
:104A50008E5B994FFC01A591B4918C9120E030E0E0
:104A6000802311F021E030E0C9011F910F910895DA
:104A700008951F920F920FB60F920BB60F9211244A
:104A80002F933F934F938F939F93EF93FF93409177
:104A9000C6002091AF223091B0222F5F3F4F2F737D
:104AA00030708091B1229091B2222817390759F0C5
:104AB000E091AF22F091B022E159FD4D4083309357
:104AC000B0222093AF22FF91EF919F918F914F9150
:104AD0003F912F910F900BBE0F900FBE0F901F9024
:104AE000189508951F920F920FB60F920BB60F9262
:104AF00011242F933F934F938F939F93EF93FF93A3
:104B00004091CE0020913723309138232F5F3F4FC3
:104B10002F7330708091392390913A2328173907E9
:104B200059F0E0913723F0913823E950FD4D40834F
:104B30003093382320933723FF91EF919F918F91EA
:104B40004F913F912F910F900BBE0F900FBE0F9082
:104B50001F901895E0918B23F0918C23E05CFF4F20
:104B60008191919120813181821B930B8F73907081
:104B7000892B11F00E943825E091AA23F091AB23F4
:104B8000E05CFF4F8191919120813181821B930BD9
:104B90008F739070892B11F00E94712508951F92D8
:104BA0000F920FB60F920BB60F9211242F933F93D3
:104BB0004F935F936F937F938F939F93AF93BF9325
:104BC000EF93FF932091F3223091F4228091F5220C
:104BD0009091F6222817390731F48091C1008F7D1A
:104BE0008093C10016C0E091F522F091F622ED54B9
:104BF000FD4D40818091F5229091F622019660E46E
:104C000070E00E94412B9093F6228093F52240930E
:104C1000C600FF91EF91BF91AF919F918F917F91CE
:104C20006F915F914F913F912F910F900BBE0F901D
:104C30000FBE0F901F9018951F920F920FB60F92F4
:104C40000BB60F9211242F933F934F935F936F9363
:104C50007F938F939F93AF93BF93EF93FF93209195
:104C60007B2330917C2380917D2390917E23281794
:104C7000390731F48091C9008F7D8093C90016C037
:104C8000E0917D23F0917E23E55CFC4D4081809195
:104C90007D2390917E23019660E470E00E94412B79
:104CA00090937E2380937D234093CE00FF91EF91DC
:104CB000BF91AF919F918F917F916F915F914F9134
:104CC0003F912F910F900BBE0F900FBE0F901F9032
:104CD0001895DC011C96ED91FC911D97E05CFF4F4F
:104CE0002191319180819181281B390B2F73307074
:104CF000C9010895DC011C96ED91FC911D97E05CC3
:104D0000FF4F20813181E054F040DF01AE5BBF4FA7
:104D10008D919C9111972817390719F42FEF3FEFC8
:104D200007C08D919C91E80FF91F8081282F30E0FA
:104D3000C9010895DC011C96ED91FC911D97E05C82
:104D4000FF4F20813181E054F040DF01AE5BBF4F67
:104D50008D919C9111972817390719F42FEF3FEF88
:104D600010C08D919C911197E80FF91F20818D91B2
:104D70009C91119701968F73907011969C938E93CE
:104D800030E0C9010895FC0186859785DC01A05CAF
:104D9000BF4FFC01EE5BFF4F2D913C91119780813D
:104DA000918128173907C1F70895CF93DF93EC015C
:104DB000462FEE85FF85E05CFF4F80819181E054B6
:104DC000F040019660E470E00E94412B9C01DF01FD
:104DD000AE5BBF4F8D919C91119728173907D1F386
:104DE000E05CFF4F80819181E054F040E80FF91FB3
:104DF0004083EE85FF85E05CFF4F31832083EE89A1
:104E0000FF89208181E090E00D8C02C0880F991FFE
:104E10000A94E2F7282B208381E090E0DF91CF9184
:104E200008951F93109282231092812328EE33E07D
:104E300040E050E0209383233093842340938523E4
:104E40005093862360E271E07093802360937F2308
:104E50008FE692E290938C2380938B2383EB92E2F4
:104E600090938E2380938D2385EC90E090939023F4
:104E700080938F2384EC90E09093922380939123EE
:104E800080EC90E0909394238093932381EC90E0C6
:104E9000909396238093952386EC90E090939823AB
:104EA0008093972314E010939923B3E0B0939A234F
:104EB000A7E0A0939B23F5E0F0939C23E1E0E0932F
:104EC0009D231092A1231092A0232093A22330931C
:104ED000A3234093A4235093A52370939F2360930F
:104EE0009E2387EF92E29093AB238093AA238BE3D8
:104EF00093E29093AD238093AC238DEC90E090935C
:104F0000AF238093AE238CEC90E09093B1238093F9
:104F1000B02388EC90E09093B3238093B22389EC84
:104F200090E09093B5238093B4238EEC90E090931F
:104F3000B7238093B6231093B823B093B923A093DB
:104F4000BA23F093BB23E093BC231F910895CF9322
:104F5000DF930E9489230E947B05CAEAD5E20E9462
:104F6000D4072097E1F30E94AA25F9CFCF92DF92D0
:104F7000EF92FF920F931F93CF93DF937C016B010E
:104F80008A01C0E0D0E00FC0D6016D916D01D7015C
:104F9000ED91FC910190F081E02DC7010995C80FBA
:104FA000D91F015010400115110571F7CE01DF9195
:104FB000CF911F910F91FF90EF90DF90CF900895C8
:104FC000813051F0813028F0823061F08330E9F493
:104FD0001AC010926E00089580916F008D7F8093AB
:104FE0006F000895809170008D7F8093700081E044
:104FF0008093B0008091B100887F84608093B1007D
:105000001092B30008951092710008951F93182F05
:1050100080911301811711F09FEF06C0ECEAF6E0D2
:1050200094918FEF80931301892F0E94E027812FA5
:1050300060E00E94D5241F9108951F920F920FB631
:105040000F920BB60F9211242F933F934F935F93C0
:105050006F937F938F939F93AF93BF93EF93FF9340
:105060008091CB239091CC23A091CD23B091CE23DE
:105070000097A105B10551F1E091CF23F091D02324
:1050800080819091D123892780838091CB23909137
:10509000CC23A091CD23B091CE23181619061A0661
:1050A0001B06C4F48091CB239091CC23A091CD23F7
:1050B000B091CE230197A109B1098093CB2390939E
:1050C000CC23A093CD23B093CE2304C080911301B1
:1050D0000E940628FF91EF91BF91AF919F918F9110
:1050E0007F916F915F914F913F912F910F900BBEE8
:1050F0000F900FBE0F901F9018952F923F925F92C6
:105100006F927F928F929F92AF92BF92CF92DF92D7
:10511000EF92FF920F931F93DF93CF9300D000D0B5
:10512000CDB7DEB7A82F1B0129833A834B835C835D
:10513000809113018A1721F4ECEAF6E05490AFC095
:105140008F3F09F02BC2A0931301ECEAF6E05490D4
:105150002FEF521609F422C281E0581671F185151D
:105160001CF0552051F09BC092E0591609F44BC039
:10517000B3E05B1609F093C06CC014BC15BC84B5D9
:10518000826084BD85B5816085BD2A2F30E0F9013C
:10519000E45BF94FE491F0E0EE0FFF1FE85CF94F9C
:1051A000859194919093C2238093C1232459394FC0
:1051B000F90184918093C32374C0109280001092EF
:1051C00081008091810088608093810080918100BE
:1051D0008160809381002A2F30E0F901E45BF94F70
:1051E000E491F0E0EE0FFF1FE85CF94F8591949198
:1051F0009093C9238093C8232459394FF90184918E
:105200008093CA234EC01092B0001092B1008091DA
:10521000B00082608093B0008091B1008160809383
:10522000B1002A2F30E0F901E45BF94FE491F0E09E
:10523000EE0FFF1FE85CF94F859194919093D02376
:105240008093CF232459394FF90184918093D1233E
:1052500028C0109290001092910080919100886077
:1052600080939100809191008160809391002A2F1A
:1052700030E0F901E45BF94FE491F0E0EE0FFF1F3D
:10528000E85CF94F859194919093D7238093D6232E
:105290002459394FF90184918093D82302C057FCD7
:1052A0007DC18A2F61E00E947124552021F0F2E037
:1052B0005F1609F0BEC031018824992460E072E1D4
:1052C0008AE790E0A40193010E94762B59016A01BC
:1052D000860175010894E108F108010911092FEF11
:1052E000E216F1040105110509F008F499C060E423
:1052F00072E48FE090E0A40193010E94762B790183
:105300008A010894E108F1080109110982E05816A0
:10531000C1F49FEFE916F1040105110509F008F445
:1053200084C060E970ED83E090E0A40193010E94E5
:10533000762B79018A010894E108F1080109110925
:1053400083E0AFEFEA16F1040105110509F008F456
:1053500068C068E478EE81E090E0A40193010E94C7
:10536000762B79018A010894E108F10801091109F5
:10537000552011F483E01DC0B2E05B1611F084E00B
:1053800018C0EFEFEE16F1040105110509F008F45D
:1053900003C164E274EF80E090E0A40193010E94F5
:1053A000762B79018A010894E108F10801091109B5
:1053B00085E0FFEFEF16F1040105110591F188F189
:1053C00062E17AE780E090E0A40193010E94762BED
:1053D00079018A010894E108F108010911095520B1
:1053E00011F086E001C084E02FEFE216F104010520
:1053F0001105B9F0B0F0C601B50120E034E040E09D
:1054000050E00E94762B79018A010894E108F108A6
:1054100001091109552011F087E008C085E003C09B
:1054200081E0552019F485BD44C082E08093B1002D
:1054300040C05101CC24DD2460E072E18AE790E0B5
:10544000A60195010E94762B79018A010894E10852
:10545000F1080109110980E0E81680E0F80681E012
:10546000080780E0180710F491E010C068E478EEB7
:1054700081E090E0A60195010E94762B79018A01D6
:105480000894E108F1080109110993E0A1E05A1616
:1054900039F480918100887F982B9093810009C016
:1054A000B3E05B1631F480919100887F982B909344
:1054B000910089819A81AB81BC810097A105B105DA
:1054C00029F48FEF9FEFAFEFBFEF13C0220C331C17
:1054D000B10180E090E029813A814B815C810E949A
:1054E0000E2B28EE33E040E050E00E94542BC9011F
:1054F000DA01E1E05E16E1F0E5151CF0552049F017
:105500004DC0F2E05F1631F123E0521609F046C0BB
:1055100031C0E7BC8093BD239093BE23A093BF23EB
:10552000B093C02380916E00826080936E0036C07D
:10553000F0928900E09288008093C4239093C52361
:10554000A093C623B093C72380916F00826080939D
:105550006F0024C0E092B3008093CB239093CC23C0
:10556000A093CD23B093CE2380917000826080936E
:10557000700014C0F0929900E09298008093D223BA
:105580009093D323A093D423B093D523809171001B
:1055900082608093710002C084E048CF0F900F902A
:1055A0000F900F90CF91DF911F910F91FF90EF908F
:1055B000DF90CF90BF90AF909F908F907F906F9033
:1055C0005F903F902F900895EF92FF920F931F935B
:1055D0007B018C01611571058105910529F420E09D
:1055E00030E040E050E00BC00E94DB04A8019701CE
:1055F0000E94762BAC01CB01DA019C01AD01B9010F
:10560000CA011F910F91FF90EF900895009729F024
:10561000BC0180E090E00E94E0040895629FD00108
:10562000739FF001829FE00DF11D649FE00DF11D5D
:10563000929FF00D839FF00D749FF00D659FF00D0C
:105640009927729FB00DE11DF91F639FB00DE11DF9
:10565000F91FBD01CF0111240895AA1BBB1B51E105
:1056600007C0AA1FBB1FA617B70710F0A61BB70BD2
:10567000881F991F5A95A9F780959095BC01CD0177
:10568000089597FB092E07260AD077FD04D0E5DFA1
:1056900006D000201AF4709561957F4F0895F6F7B3
:1056A000909581959F4F0895A1E21A2EAA1BBB1BCE
:1056B000FD010DC0AA1FBB1FEE1FFF1FA217B307DE
:1056C000E407F50720F0A21BB30BE40BF50B661FF4
:1056D000771F881F991F1A9469F7609570958095B8
:1056E00090959B01AC01BD01CF01089597FB092E58
:1056F00005260ED057FD04D0D7DF0AD0001C38F4A1
:1057000050954095309521953F4F4F4F5F4F0895ED
:10571000F6F790958095709561957F4F8F4F9F4FCD
:105720000895EE0FFF1F0590F491E02D09942F923C
:105730003F924F925F926F927F928F929F92AF9221
:10574000BF92CF92DF92EF92FF920F931F93CF936E
:10575000DF93CDB7DEB7CA1BDB0B0FB6F894DEBF05
:105760000FBECDBF09942A88398848885F846E842B
:105770007D848C849B84AA84B984C884DF80EE8075
:10578000FD800C811B81AA81B981CE0FD11D0FB67E
:10579000F894DEBF0FBECDBFED010895F894FFCFA2
:1057A0002000DD230000010000006B146B14FFFFDC
:1057B000FFFF01FF000000003520B62700000000B9
:0C57C000D526B62769269A267A26C3262D
:00000001FF
